S01F00006F70656E626C745F6F6C696D6578696E6F5F73746D33322E73726563C6
S3150800000000500020C950000819510008195100086D
S31508000010195100081951000819510008000000007C
S315080000200000000000000000000000001951000850
S31508000030195100080000000019510008195100085C
S3150800004019510008195100081951000819510008DA
S3150800005019510008195100081951000819510008CA
S3150800006019510008195100081951000819510008BA
S3150800007019510008195100081951000819510008AA
S31508000080195100081951000819510008195100089A
S31508000090195100081951000819510008195100088A
S315080000A0195100081951000819510008195100087A
S315080000B0195100081951000819510008195100086A
S315080000C0195100081951000819510008195100085A
S315080000D0195100081951000819510008195100084A
S315080000E019510008195100081951000800000000AC
S315080000F000000000000000000000000000000000F2
S3110800010000000000000000005FF808F195
S3150800010C10B5054C237833B9044B13B10448AFF337
S3150800011C00800123237010BDC002002000000000DF
S3150800012C2454000808B5034B1BB103490348AFF325
S3150800013C008008BD00000000C402002024540008FA
S3150800014C72B6704762B67047FFF7FABF10B500F083
S3150800015C9DFA00B910BD03F0EDF90028FAD000F0AD
S3150800016CFFFC00F0B5FA00F093FA074B20F060405C
S3150800017C20F07F00186000F08BFA4468FFF7E2FF66
S3150800018C2346BDE81040184708ED00E072B170B57B
S3150800019C0D46561EB6B20644441E15F8013B04F825
S315080001AC013F00F005FDB442F7D170BD704700BFA2
S315080001BC2DE9F041DFF83C800746464600250C4CF5
S315080001CC01E056F80C4F00F0F3FCBC4203D87368F8
S315080001DC1C44A74205D301350D2DF2D1FF20BDE8ED
S315080001ECF08105EB450508EB8505287ABDE8F08115
S315080001FC006000083C5400082DE9F047804600686A
S3150800020CFFF7D6FFFF285ED03422314B31483249EE
S3150800021C58605960DA60DD6815F001053FD14FF07A
S3150800022C01091C461A6942EA09021A612F1D58F877
S3150800023C0760D8F80030B2B2EA521D4400F05CFAF6
S3150800024C00F1050A05E000F0B3FC00F055FA82450A
S3150800025C2ED3E368DA07F6D4330C6B8000F04CFA2D
S3150800026C00F1050A05E000F0A3FC00F045FA82450A
S3150800027C21D3E368DB07F6D42B689E4220D1B7F569
S3150800028C007F3D46D2D1124B48461A6922F001022C
S3150800029C1A611A6942F080021A61BDE8F0874FF0BC
S315080002AC00091A69484642F080021A61BDE8F087CF
S315080002BC4FF00009D0E72B684FF000099E42DED0BC
S315080002CC4FF00009DFE74FF000094846BDE8F08714
S315080002DC0020024023016745AB89EFCD70B5104C61
S315080002EC0D46A0421AD00F4B99420AD00646FFF784
S315080002FC83FF10B1C5F3080313B10024204670BD63
S3150800030C34462368AB42F9D02046294640F8045BAC
S3150800031C4FF40072FFF73AFF204670BD024EE9E72C
S3150800032CE004002000600008DC0200202DE9F843F8
S3150800033C0C46016824F4FF781D464B1C07461646E6
S3150800034C28F0010832D0884506D038464146FFF7D2
S3150800035CC5FF074638B301680434641A3C4408F5EB
S3150800036C007807F1040905E016F8013B013D04F88D
S3150800037C013B15D000F01CFCA4EB0903B3F5007F78
S3150800038CF2D338464146FFF7A9FF074600F10409A0
S3150800039C48B14C4616F8013B013D04F8013BE9D13E
S315080003AC0120BDE8F8830020BDE8F883814649F8AA
S315080003BC048B414648464FF40072FFF7E7FE39684E
S315080003CCC1E700BF4FF0FF330249034A0B601360C5
S315080003DC704700BFDC020020E0040020FFF7F2BFE4
S315080003EC70B5144C4B1E241AA34201D9002070BDBB
S315080003FC054616460C46FFF7DBFEFF28F6D0681EA8
S3150800040C2044FFF7D5FEFF28F0D00B4A25F4FF73DE
S3150800041C23F00103934229462346324604D0BDE80D
S3150800042C70400648FFF782BF0548BDE87040FFF7E5
S3150800043C7DBF00BFFFFF010800600008DC0200203A
S3150800044CE0040020574B2DE9F0471B1A4C1E9C4222
S3150800045C03D900263046BDE8F08704460D46FFF75B
S3150800046CA7FE0646601E2844FFF7A2FE86420446EF
S3150800047CEFD8F31EDBB2FB2BEBD80F28E9D83423C5
S3150800048C494A4A484A4950605160D360D56815F0C4
S3150800049C01056ED11369474F43F00203B846B946B6
S315080004AC4FF0030A136101E099F808A000F080FBED
S315080004BC564509F10C0962D001350D2DF4D14FF0D2
S315080004CCFF3500264FF0030ADFF8E89001E099F8AB
S315080004DC08A000F06DFB544509F10C095CD00136F7
S315080004EC0D2EF4D14FF0FF3900264FF0030A01E028
S315080004FC97F808A000F05CFB544507F10C0744D0AC
S3150800050C01360D2EF4D10022A9EB05031344C3F3CF
S3150800051C8F2301261BB303F1FF381FFA88F805F55C
S3150800052C8067214C07EB88286561236943F04003F3
S3150800053C236100F0E1F800F1640505E000F038FBF2
S3150800054C00F0DAF8854208D3E368DB07F6D4B84539
S3150800055C3D4604D007F58067E6E70026F7E7124B19
S3150800056C1A6922F002021A611A6942F080021A61AB
S3150800057C70E71369002643F0800313616AE7EDB24E
S3150800058C05EB450558F825509BE7F6B206EB4606EB
S3150800059C08EB86067268B7E7F6B206EB460658F815
S315080005AC2690A1E7FFFF01080020024023016745BA
S315080005BCAB89EFCD3C5400080F490B68013318D0B2
S315080005CC88684B6810B5CC680344086923444C69A1
S315080005DC034488692344C969034482B00B4402AABC
S315080005EC5B4242F8043D04210448FFF7F9FE02B0C9
S315080005FC10BD0120704700BFE00400200C61000804
S3150800060C0D4A0E4B0E4910681B6810B40C6803444F
S3150800061C906823448C68034410311069234402F50E
S3150800062C84720968034412680B44D3420CBF012038
S3150800063C002010BC704700BF04600008006000086A
S3150800064C086000080A4808B50368013302D0FFF7AA
S3150800065CD3FD58B107480368013305D0FFF7CCFD25
S3150800066C003018BF012008BD012008BD08BD00BF19
S3150800067CE0040020DC0200200048704700600008F7
S3150800068CFFF7ACBEFFF7ACBEFFF7DCBEFFF7B8BF93
S3150800069CFFF7F2BF08B5FFF78FFF00B908BDBDE835
S315080006AC0840FFF7CFBF00BF0022052010B4054B4A
S315080006BC054C06491A605C609A6010BC18600A60A2
S315080006CC704700BF10E000E03F190100E406002067
S315080006DC0022014B1A60704710E000E0044B1B68BF
S315080006ECDB0303D5034A136801331360704700BF55
S315080006FC10E000E0E4060020044B1B6813F4803F6E
S3150800070C034B18681CBF01301860704710E000E0F6
S3150800071CE4060020B2B1002370B41E46541EE4B29F
S3150800072C01346400020F092A02F1300586BF3732FC
S3150800073CCA54CD54CA1802339C424FEA001056705C
S3150800074CF0D170BC704700BF012838B504460D4679
S3150800075C04D94FF4FA710F4800F082F904EB4404FB
S3150800076C0D48E4000319597C1A7C914210D0DA68BA
S3150800077C1570DA68597C5D6801320131AA425974E0
S3150800078CDA6003D902590120DA6038BD012038BD78
S3150800079C002038BDD854000868070020012870B519
S315080007AC04460E4604D940F216210E4800F058F9B4
S315080007BC04EB44040C4DE4002B19587C80B19A6860
S315080007CC127832709A68597C58680132013982421B
S315080007DC59749A6003D92A5901209A6070BD012070
S315080007EC70BD00BFD854000868070020F0B4402537
S315080007FC01260022114B124C124903F118005861BC
S3150800080C601958604819104FD861A0199860D860BB
S3150800081C18609A7488195A7483F829200E7083F80C
S3150800082C2A601D7483F8285022703A60DA621862BE
S3150800083C58629861F0BC03F093BC00BF68070020AF
S3150800084C9C070020E007002098070020002002F0F3
S3150800085C3DBE00BF3F29F8B50D46044621D8134EB8
S3150800086C29463078FFF770FF012803D096211048E7
S3150800087C00F0F6F8ADB29DB1013DADB20C4F254472
S3150800088C013C00F095F914F8011F3078FFF75CFF6E
S3150800089C012803D09F21384600F0E2F8AC42F0D18B
S315080008ACF8BD9221024800F0DBF8D8E79C07002037
S315080008BCD85400082DE9F8431C4D80460F4604F021
S315080008CC35FC2C785CB91A4B1A4E18783146FFF75A
S315080008DC65FF012822D000242046BDE8F883164E71
S315080008EC134B3178DFF84C90013149441878FFF7EF
S315080008FC55FF01280446EED1337899F800200133C8
S3150800090CDBB29A423370E6D109F101014046FFF792
S3150800091C3DFC002233782A703B70DDE73378013BC7
S3150800092C3E2BD8D8044B28701C70D5E764080020D9
S3150800093CE007002024080020650800202DE9F04176
S3150800094C1E4F82B03C78012C04D940F236211C4843
S3150800095C00F086F81B4B04EB440403EBC404667CDA
S3150800096C46B3402E28BF40260024174DDFF850808A
S3150800097C0DF107013878FFF711FF012804D040F272
S3150800098C4511404600F06CF801349DF80730E4B286
S3150800099CA64205F8013FEBD8B6B232464FF4807141
S315080009AC0A4803F0B9FC0120314603F081FD012009
S315080009BC03F020FD02B0BDE8F08100BF9C070020C3
S315080009CCD8540008680700202707002028070020AD
S315080009DCF8B5104C0120214603F008FE80B298B1F8
S315080009EC451EADB20C4E0D4F2544013C14F8011FA3
S315080009FC3078FFF7A9FE012804D04FF4B5713846B4
S31508000A0C00F02EF8AC42F1D10120BDE8F84003F015
S31508000A1C05BD00BFE8060020E0070020D8540008F2
S31508000A2C0A490B4A0B4B086810B514681B68C018A2
S31508000A3C00D110BD08220849FFF76CFE2046BDE818
S31508000A4C104004220549FFF765BE00BFE8F7FF1FF3
S31508000A5CECF7FF1FF0F7FF1F06000020160000201A
S31508000A6C08B500F0A5F8FCE710B500F09DF80128CC
S31508000A7C06D000F009F918B10B4C2378012B00D0DD
S31508000A8C10BDFFF739FE094B1B6803F5FA6398424C
S31508000A9CF6D30023237000F0FFF80028F0D1BDE848
S31508000AAC1040FFF753BB00BF6608002068080020FB
S31508000ABC012208B5044B1A70FFF71EFE034B18608B
S31508000ACCBDE80840FFF7D0BF66080020680800207C
S31508000ADC08B5FFF739FB00F069F8FFF7E5FDFFF7F6
S31508000AECCFFD00F0B7F800F013F8BDE80840FFF7A3
S31508000AFCDFBF00BF08B500F05BF8FFF7EFFD00F0AD
S31508000B0CDDF900F011F8BDE80840FFF7ADBF00BFEE
S31508000B1C08B502F04BFBFFF769FE0222014B1A706F
S31508000B2C08BD00BF0000002000B583B00DF1070119
S31508000B3C0948FFF7BFFE012802D003B05DF804FB95
S31508000B4C0222064B9DF8071003481A7002F04CFB5C
S31508000B5C03B05DF804FB00BF6C0800200000002001
S31508000B6CFFF774BE08B5074B1B78022B03D0BDE8FC
S31508000B7C084002F031BBC9B2FFF76CFEBDE808406D
S31508000B8C02F02ABB00000020044B1B78032B9ABFEB
S31508000B9C034A32F813003F20704700BF00000020BC
S31508000BAC00550008FFF7F0BF02F00EBB02F0CEBCF2
S31508000BBC02F0D0BC092800F00F0302D903F1370064
S31508000BCC704710B503F1300404F0F0FB2044437869
S31508000BDC03F00303022B14BF2046A4F12000C0B275
S31508000BEC10BD00BF38B5054600090C46FFF7E2FFF5
S31508000BFC207005F00F00FFF7DDFF00236070A3706F
S31508000C0C204638BDF8B50027461E451C16F8014F78
S31508000C1C04F0CCFB2044417801F00301022908BFFB
S31508000C2C203CE3B2A3F13002D2B2162AA3F13A0160
S31508000C3C0DD806290BD9092A84BF373BDAB202EB41
S31508000C4C0713AE4203F0FF07E0D13846F8BD00277C
S31508000C5C3846F8BD002310B5074C1A46074908480C
S31508000C6C237001F095FD00B910BD7721BDE8104041
S31508000C7C0448FFF7F5BE00BF0C0D00200855000808
S31508000C8CB40800200C550008024B1878B0FA80F00E
S31508000C9C400970470C0D002010B5FFF785FF012899
S31508000CAC02D0054C23780BB1002010BD02F054FC81
S31508000CBC0128F9D1207010BD0C0D002038B5054659
S31508000CCC047804F073FB2044437803F00303022BE7
S31508000CDC08BF203C532C01D0032038BD04F066FB1A
S31508000CEC6B78184442785207F6D5312B05D0322B3F
S31508000CFC05D0332BF0D1022038BD002038BD012099
S31508000D0C38BD00BF70B506460230FFF77BFF0546B7
S31508000D1C043684B23046FFF775FF013CA4B205448D
S31508000D2C012CEDB206F10206F4D83046ED43FFF776
S31508000D3C69FFEDB2281AB0FA80F0400970BD00BF01
S31508000D4C2DE9F041044617468846002951D000285B
S31508000D5C4FD02046FFF7B2FF0328054645D020465C
S31508000D6CFFF7D0FF002800F0A380012D47D078D3D9
S31508000D7C022D3AD1A01CFFF745FF0546201DFFF7AB
S31508000D8C41FF0006C8F80000A01DFFF73BFFD8F886
S31508000D9C0030053D03EB0040C8F8000004F10800DC
S31508000DACFFF730FFD8F8003004F10C0603EB0020EF
S31508000DBCC8F8000004F10A00FFF724FFD8F8003041
S31508000DCC2DB20344C8F8003087B1002D0EDD00247F
S31508000DDC3046FFF717FF631C38559CB2AC4206F138
S31508000DEC0206F5DB2846BDE8F08100252846BDE855
S31508000DFCF08140F261213048FFF732FEA9E7A01CCA
S31508000E0CFFF700FF0546201DFFF7FCFE0004C8F897
S31508000E1C0000A01DFFF7F6FED8F80030043D03EBE2
S31508000E2C0020C8F8000004F10800FFF7EBFED8F81C
S31508000E3C003004F10A0603442DB2C8F80030002F1E
S31508000E4CD4D0002DD2DD00243046FFF7DBFE631C20
S31508000E5C38559CB2AC4206F10206F5DB2846BDE8CD
S31508000E6CF081A01CFFF7CEFE0546201DFFF7CAFE33
S31508000E7C0002C8F80000A01DFFF7C4FED8F8003021
S31508000E8C033D03442DB20834C8F80030002FADD00A
S31508000E9C002DABDD00262046FFF7B4FE731CB855B3
S31508000EAC9EB2AE4204F10204F5DB2846BDE8F08199
S31508000EBC4FF0FF359AE700BF0C5500082DE9F843AB
S31508000ECCAA4F3C783CB1012C00F01781022C00F09B
S31508000EDC8E80032C01D0BDE8F883A54EA54D06F5EA
S31508000EEC0C7228464FF4807102F09AF896F84192E3
S31508000EFCB9F1000F40F0BA81002855D005F580727B
S31508000F0C05F5C0712846FFF71BFFB0F1FF3F804679
S31508000F1C00F01E81002847DD974802F073FB434614
S31508000F2C9649974AA2FB0303DB0801F10101F9D1A3
S31508000F3C444693480B70A0FB0423DB0803EB83029F
S31508000F4CA4EB4202303201F8012D1C46002BF2D1DB
S31508000F5C8A4802F057FB8B4802F054FB874995F8F0
S31508000F6C8301FFF73FFE884995F88201FFF73AFEA1
S31508000F7C864995F88101FFF735FE854995F8800174
S31508000F8CFFF730FE7D4802F03DFB824802F03AFB43
S31508000F9C4146D5F88001804AFFF774FB002800F01B
S31508000FAC75817E4802F02EFBD6F84422D6F83C32E0
S31508000FBC9A4290D17A4802F025FBFFF76BFB044660
S31508000FCC002800F07C81754802F01CFB754802F07D
S31508000FDC19FB754801F0D4FE744802F013FB002384
S31508000FEC3B7002F0EFFABDE8F843FFF7AFB8604E76
S31508000FFC604D06F50C7228464FF4807102F010F815
S3150800100C96F84192B9F1000F40F03E81D0B14A46AC
S3150800101C05F5C0712846FFF793FEB0F1FF3F8046F1
S3150800102C00F0598100280DDD614C6368002B00F037
S3150800103C18812268D5F880111A44914240F0CA806A
S3150800104C03446360D6F84422D6F83C329A427FF4BD
S3150800105C42AF0021544801F0A5FE002840F03D811E
S3150800106C534C6368002B41D04C4802F0CBFA5148DC
S3150800107C02F0C8FA636841491A464148A0FB025275
S3150800108CD20801F10101F9D13D4D0A70A5FB030205
S3150800109CD20802EB8200A3EB4003303301F8013D82
S315080010AC1346002AF2D1354802F0ACFA424802F04F
S315080010BCA9FA3249E078FFF795FD3349A078FFF78E
S315080010CC91FD32496078FFF78DFD31492078FFF79D
S315080010DC89FD2A4802F096FA2E4802F093FA94E80B
S315080010EC0300FFF7D1FA002800F0DC802B4802F049
S315080010FC89FA03233B70BDE8F883FFF7C1FA02F0BF
S3150800110C4DFA2E4802F07EFA2D4802F07BFA02F0D0
S3150800111C41FA22460146244801F068FB054638B1D7
S3150800112C284802F06FFA2046BDE8F84302F060BA88
S3150800113C1A4802F067FA244802F064FA234802F0C7
S3150800114C61FA02221A4B3A701D605D60BDE8F8839D
S3150800115C1F4802F057FA032002F04AFA06F50C70FB
S3150800116C01F00EFE87F80090BDE8F8830C0D002000
S3150800117CB4080020100D002048560008940E0020D4
S3150800118CCDCCCCCC58560008960E0020980E0020D4
S3150800119C9A0E002088560008100E00207C55000870
S315080011AC705600088C560008E40A0020A45600085D
S315080011BCAC080020D8550008E45500082855000846
S315080011CC4C5500087455000884550008A8550008A5
S315080011DC24560008434802F015FA434802F012FA5E
S315080011EC636842491A464248A0FB02E2D20801F15A
S315080011FC0101F9D1DFF8F8E00A70AEFB0302D20858
S3150800120C02EB8200A3EB4003303301F8013D134691
S3150800121C002AF2D1354802F0F5F9364802F0F2F90F
S3150800122C3249E078FFF7DEFC3349A078FFF7DAFCA1
S3150800123C32496078FFF7D6FC31492078FFF7D2FCA3
S3150800124C2A4802F0DFF92F4802F0DCF994E803008B
S3150800125CFFF71AFA30B3234802F0D4F92A4802F0F9
S3150800126CD1F9D5F8803184E80801EBE6274802F075
S3150800127CC9F9022002F0BCF906F50C7001F080FDE4
S3150800128C00233B70BDE8F8832148F0E7204802F0BC
S3150800129CB9F9062002F0ACF91E4801F071FD3C7054
S315080012ACBDE8F8831A4802F0ADF9052002F0A0F95A
S315080012BC184801F065FD00233B70BDE8F883144817
S315080012CC02F0A0F9072002F093F9124801F058FD34
S315080012DC3C70BDE8F8830E483BE70D4802F092F9DE
S315080012EC0420E3E77C550008D8550008940E002026
S315080012FCCDCCCCCCE4550008960E0020980E0020D8
S3150800130C9A0E002088560008A855000800560008B2
S3150800131C74550008E40A002030B40468D4B1257862
S3150800132C1F2D0AD93A2D15D0234602E03A2A07D0A2
S3150800133C0B465A78591C1F2AF8D8002030BC70471F
S3150800134C0134A14206D1302D04D130BC02330360DE
S3150800135C002070474FF0FF3030BC704758B110B5BD
S3150800136C036882B004460BB11A7842B900230920E7
S3150800137C0B6002B010BD002309200B607047D8889B
S3150800138CA2889042F2D15878019103F08FFB10F0A5
S3150800139C01000199EAD123680B60EAE70B4610B401
S315080013AC0A44013813F8014B934200F8014FF9D15E
S315080013BC10BC7047F8B5C46A00F1300705462246DA
S315080013CC39464078012303F0CBFBB0B92A6AAB69DE
S315080013DCA21A9A42E8700ED2AE78012E01D80AE00B
S315080013ECAB691C44013E224601233946687803F052
S315080013FCB7FB012EF4D10020F8BD0120F8BD00BFC3
S3150800140C38B5C36A8B4217D0C37804460D4673B9F0
S3150800141C2A46012304F13001607803F051FB0028B9
S3150800142C16BF4FF0FF3500200120E56238BDFFF7E7
S3150800143CC1FF0028ECD038BD002038BD2DE9F84393
S3150800144CC378054663B92B78032B0FD0002268782E
S3150800145C114603F0EBFB003018BF0120BDE8F883FA
S3150800146CFFF7A8FF0028EED0BDE8F8832B79012BEF
S3150800147CECD105F130010B46002405F50C7203F886
S3150800148C014B9342FBD14FF0520E72204FF0AA0C2F
S3150800149C612741264FF055082B6985F814021A0A5C
S315080014AC85F8183285F819224FEA13491A0EEB6893
S315080014BC85F81B221A0A85F81C3285F81D221A0C87
S315080014CC1B0E85F81F32EB6985F81E225A1C85F807
S315080014DC150285F81A9285F82E82EA6285F82FC2CB
S315080014EC85F830E085F831E085F8327085F81772A2
S315080014FC85F8336085F816620123687803F030FBAB
S3150800150C2C71A3E700224FF0FF3310B5C270C362EB
S3150800151C0446FFF775FF08B1042010BD4AF655229C
S3150800152C94F82F1294F82E3243EA0123934201D0F1
S3150800153C032010BDB4F8681094F8672094F8663048
S3150800154C42EA012243EA02230A4A23F07F439342E2
S3150800155CEFD0B4F8841094F8833094F8820043EAF8
S3150800156C012340EA032020F07F40904214BF02205A
S3150800157C002010BD464154000023F0B50B6085B021
S3150800158C0F461446FFF7C8FE061E18DBC14B53F868
S3150800159C2650BDB13D602B7804F0FE0423B1687863
S315080015AC03F084FAC70710D50023F0B268702B70C5
S315080015BC03F016F9C1070ED5032005B0F0BD0B20B4
S315080015CC05B0F0BD0C2005B0F0BDB4B310F00400A6
S315080015DCF3D00A20F1E70CB14207FAD400212846C9
S315080015ECFFF790FF022806D0042824D0012840F2E1
S315080015FCCF800D20E1E76C46694605F5FC7305F5C9
S3150800160C0E7613F8062C42B11F8813F8010C13F842
S3150800161C022C40EA072042EA00221033B34241F872
S3150800162C042BEED104AF54F8046B46B90320A74239
S3150800163CF9D10428DDD10120BFE72046BDE73146A4
S3150800164C2846FFF75FFF0128F1D895F83C2095F856
S3150800165C3B3043EA0223B3F5007FCAD195F84720FD
S3150800166C95F8463053EA022340F09480B5F85610A4
S3150800167C95F8553095F8542043EA012342EA03229B
S3150800168C95F84040AA61631E012BAC70B1D895F849
S3150800169C3DE01FFA8EF36B81002BAAD00EF1FF33B7
S315080016AC13EA0E0FA5D195F8423095F8410040EA99
S315080016BC0320030728819CD195F8441095F84330EC
S315080016CC53EA012309D1B5F8527095F8511095F8DB
S315080016DC503041EA072143EA012395F83F7095F803
S315080016EC3E1051EA072184D002FB04F401EB1017D3
S315080016FC2744BB42FFF47DAFDB1BB3FBFEF3002B89
S3150800170C3FF477AF40F6F57E734540F2A3804FF66B
S3150800171CF57E734540F28380314495F85B40296227
S3150800172C95F85A100233374451EA04216B61AF62BB
S3150800173CEE617FF45EAF00287FF45BAFB5F85E40D0
S3150800174C95F85D0095F85C109B0040EA042003F2BE
S3150800175CFF1341EA0021B2EB532F6962FFF449AF3C
S3150800176C4FF0FF32802195F8610095F860302A61B8
S3150800177C43EA0023012BEA6029710DD00323464A5C
S3150800178C2B701388002001339BB21380EB8014E76F
S3150800179C00265AE71A4673E7711C2846FFF730FEEF
S315080017AC0028EBD14AF65522002095F82F1295F809
S315080017BC2E32287143EA01239342DFD1698E95F8BC
S315080017CC312095F8303042EA0122344943EA0223A3
S315080017DC8B42D3D1B5F8161295F8152295F8143212
S315080017EC42EA01222E4943EA02238B42C6D1B5F8B6
S315080017FC1A7295F81942B5F81E6295F81D0295F8F5
S3150800180C181295F81C2244EA072440EA062041EAF5
S3150800181C042142EA002203232961EA60AFE7023376
S3150800182C314437446B612962AF62EE6100283FF49C
S3150800183CE0AE5B0003F2FF132144B2EB532F69624F
S3150800184CFFF4D7AE4FF0FF3380222B61EB602A7181
S3150800185C022394E70233314437446B612962AF6241
S3150800186CEE6100283FF4C5AE03F0010000F2FF104C
S3150800187C03EB430300EB53032144B2EB532F69628A
S3150800188CFFF4B7AE4FF0FF3380222B61EB602A7161
S3150800189C012374E7D40E0020D80E00205252614161
S315080018AC72724161012919D94269F8B59142074604
S315080018BC07D202780C46022A2BD0032A10D0012A0A
S315080018CC01D00120F8BD016A04EB540601EB562140
S315080018DCFFF796FD78B34FF0FF30F8BD012070473F
S315080018EC016A01EBD411FFF78BFD0028F3D1A10097
S315080018FC01F4FE7101F130023A447B185188527892
S3150800190C93F8300042EA012340EA032020F07040A5
S3150800191CF8BD016A01EB1421FFF772FD0028DAD134
S3150800192C630003F4FF733B4493F8312093F83000BB
S3150800193C40EA0220F8BD396AC6F3080301363B446F
S3150800194C01EB5621384693F83050FFF759FD00281D
S3150800195CC1D1C6F30806BB1993F83000E30745EA6C
S3150800196C00204CBF0009C0F30B00F8BDB1F5001FF1
S3150800197C01D302207047CA06F8B50C4601D00220DE
S3150800198CF8BD816805460461076829B93B78022BBE
S3150800199C19D97B6ABBB119467E897602B44226D31D
S315080019ACA41B384608E00128E9D97B699842E6D297
S315080019BCA6421DD82868A41BFFF774FF431C0146D2
S315080019CCF1D10120F8BD3B89B3EB541FD7D97A6AFC
S315080019DCAA616961002AD2D007F13003C4F3080161
S315080019EC02EB54220B44EB61AA610020F8BD7B691B
S315080019FC023B881E98422FBF00227A89BB6A00FBDD
S31508001A0C0232AA61E5E700BF2DE9F04790F800908D
S31508001A1C0546B9F1020F0C46174655D0B9F1030F16
S31508001A2C2FD0B9F1010F03D002263046BDE8F08756
S31508001A3C016A04EB540801EB5821FFF7E1FC064652
S31508001A4C0028F2D108F1010AE307C8F30808A844EC
S31508001A5C51D598F83030284603F00F0343EA07139C
S31508001A6C88F83030296A85F8039001EB5A21FFF77C
S31508001A7CC7FC00284AD1CAF3080AAA44C7F30717B1
S31508001A8C50E0016A01EBD411FFF7BAFC06460028B0
S31508001A9CCBD10120A40004F4FE7404F130012944CE
S31508001AAC4B8827F070471B0403F070431F432C44E4
S31508001ABC84F830703A0A3B0C3F0E4A708B70CF7024
S31508001ACCE8703046BDE8F087016A01EB1421FFF790
S31508001ADC97FC06460028A8D101239C4004F4FF7401
S31508001AEC2C44C7F3072284F8307084F83120EB7045
S31508001AFC3046BDE8F08788F83070296A85F8039077
S31508001B0C01EB5A212846FFF77BFC08B106468CE701
S31508001B1CCAF3080AAA449AF83020C7F3032722F016
S31508001B2C0F02174301238AF83070EB707DE700BF6C
S31508001B3C2DE9F04107468846066849BBF56873697E
S31508001B4CF5B901252C4606E0012815D001302ED012
S31508001B5CAC4219D0736901349C4202D3012D13D9B6
S31508001B6C022421463868FFF79DFE0028ECD1012C8B
S31508001B7C02D973699C421FD301242046BDE8F08123
S31508001B8C9D4228BF0125DDE700242046BDE8F081EB
S31508001B9C3046FFF787FE01280446EDD9431C06D0CC
S31508001BAC73699842E9D34546CCE70128E4D14FF04E
S31508001BBCFF342046BDE8F0814FF0FF32214630460F
S31508001BCCFFF722FF0028F0D1B8F1000F0CD0B8F1BE
S31508001BDC010FD1D973699845CED241462246304673
S31508001BECFFF712FF0028E0D172693369023A934273
S31508001BFCF46001D2013B3361337943F0010333714D
S31508001C0CBBE700BF83690BB9042070472DE9F04781
S31508001C1C056982B02035B5F5001F03D3042002B040
S31508001C2CBDE8F087C5F308070E46044602681FBBD5
S31508001C3C41690133836129B35389013B13EA55235F
S31508001C4C1AD110460192FFF72DFE01288046019AFB
S31508001C5C20D9B0F1FF3F31D0536998421CD2861E69
S31508001C6C023B9E422EBF00265389916AC4F8148003
S31508001C7C38BF06FB0316A66130371744E7612561A2
S31508001C8C0020CCE71389B3EB551FF5D800230420A5
S31508001C9CA361C4E70220C2E7002EF7D0616920468B
S31508001CAC0192FFF745FF019A804648B90720B6E727
S31508001CBC10460192FFF77EFB019A48B10120AEE768
S31508001CCC0128E7D0B0F1FF3FF8D0D378002BEFD13D
S31508001CDC002102F50C7002F1300303F8011B98423F
S31508001CECFBD15369A8F10206023B9E4220D25189C8
S31508001CFC936A06FB0133D3624FF000094FF0010AD1
S31508001D0C0EE082F803A010460192FFF753FB002859
S31508001D1CD4D1019A09F10109D36A51890133D362E5
S31508001D2C8945EED3D16A5369A1EB0901D16297E7CC
S31508001D3C00235189DFE700BF416A2DE9F0414B1CAE
S31508001D4C04460568066904D0FFF710FE08B1BDE81D
S31508001D5CF0814FF0E50801270BE0E36983F8008072
S31508001D6CEF7023699E42F2D901462046FFF74AFFD7
S31508001D7C28B9A1692846FFF743FB0028EDD00428AB
S31508001D8C08BF0220BDE8F0812DE9F04F002185B08F
S31508001D9C06460768FFF7EAFD002852D14FF0FF33D5
S31508001DAC4FF0FF099846CA4673620BE00F2B4BD0CF
S31508001DBC4FF0FF0AC6F8248000213046FFF722FFB1
S31508001DCC00283ED1B1693846FFF71AFB002838D1EE
S31508001DDCF4692578002D00F08F80E27AE52D02F063
S31508001DEC3F03B371E4D01207E0D40F2B2CD0BAF111
S31508001DFC000F0FD1214604F10B0511F8012B4FEA00
S31508001E0CCA1343EA5A0A9244A9420AF0FF0AF4D1C1
S31508001E1CD14516D0316ACB7ADB07C9D40D4623785F
S31508001E2C15F80B2B01319B1A0134002BC0D111F874
S31508001E3C012B14F8013B8D42A3EB0203F5D1002BC1
S31508001E4CB6D105B0BDE8F08FB36A002BB4D06906DD
S31508001E5C4DD5326994F80D9005F0BF05726294F869
S31508001E6C0DB0CB4545D1E17EA27E52EA012240D186
S31508001E7C012194F800A02D4A0AF03F0A0AF1FF3A0C
S31508001E8C0AEB4A000AEB800A039591462546009709
S31508001E9C1C46CDF804B00846029613E0BAF1FE0FBC
S31508001EAC1ED8384601F02EF9834634F81A0001F08C
S31508001EBC29F9834514D13846B2461D4B4B451FD0DC
S31508001ECC19F8011F6F1897F801E06F5C0AF1010603
S31508001EDC47EA0E270028E1D14FF6FF739F42ECD054
S31508001EEC9DE88008029ED9464FF0FF0A64E7AA458A
S31508001EFCB5D04FF0FF0A5FE7042005B0BDE8F08FB8
S31508001F0C23462C462278009F5206039DDDF804B022
S31508001F1C029E03D510B133F81A3023B9013D5FFA86
S31508001F2C85FAD94648E7D946E3E700BF5057000873
S31508001F3C5C5700082DE9F04F076A89B0FB7A13F055
S31508001F4CA00304D00626304609B0BDE8F08FD0F8B9
S31508001F5C2890B9F80020002A00F0D88098464B46FD
S31508001F6C33F8022F08F10108002AF9D104460C228D
S31508001F7C05A83946D4F800B0FFF710FA9DF81F30BB
S31508001F8CDD076DD500234FF0010AFB720B22A36205
S31508001F9C05A93846FFF702FA53469B4D07220DF161
S31508001FAC130603F00F0000F13001392988BF00F140
S31508001FBC37011B0902F1FF3206F80119F1D17E200F
S31508001FCC08A9114401F8140C5AB13978202909D0FA
S31508001FDC394603E011F8010F202803D001339A4241
S31508001FECF8D113463B44072A08A911448EBF202171
S31508001FFC11F8141C013203F8011BD91B0729F2D955
S3150800200C2046FFF7C1FE064600BB0AF1010ABAF1E3
S3150800201C640F76D00B2205A93846FFF7BFF9BAF13B
S3150800202C050F5346BAD9A9F1020636F8022F002A2B
S3150800203CB4D0102102F0010000EB4303D80348BFCB
S3150800204C6B4001394FEA5202F4D1EEE704287FF4CB
S3150800205C7AAF9DF81F30FB729DF81F30C4F8289094
S3150800206C9B0742D4012700212046D4F80080FFF7AD
S3150800207C7DFC0646002841D1054606E005460121A9
S3150800208C2046FFF7BFFD002837D1A1694046FFF768
S3150800209CB7F9013588BBE3691B78E52B01D0002B12
S315080020ACECD1AF42EBD1B7F1010A31D1A16958464F
S315080020BCFFF7A6F9064600287FF445AF3146E369D3
S315080020CC03F1200203F8011B9A42FBD10B22216A69
S315080020DCE069FFF763F90122236AE169DB7A03F009
S315080020EC18030B738BF803202DE7484B08F10C07E4
S315080020FCA3FB0737BF080137B5E70646042E7FF45E
S3150800210C22AF0726304609B0BDE8F08F90462DE77A
S3150800211C21692046A1EB4A11FFF728FC0646002840
S3150800212C7FF411AF216A814608460B314FEAC91371
S3150800213C10F8012B43EA59031344884203F0FF09AC
S3150800214CF4D1DFF8CC80A1695846FFF759F9034654
S3150800215C002857D15FFA8AFC0CF1FF3505EB4502CE
S3150800216C05EB820505F10046A26A013E019202EBD7
S3150800217C46064FF00F02E16908738876C876012087
S3150800218CCA72234A81F80D90009236F8022F0F185E
S3150800219C4FEA122E0A54013587F801E00133E2B9E9
S315080021AC0D2B0AD0FF22013B434413F8010F0D18DF
S315080021BC0A5418486A709842F7D14CF0400C01231F
S315080021CC81F800C0204600218BF80330FFF71AFD72
S315080021DCC0B9BAF1010AB6D168E70D2B08D04FF68B
S315080021ECFF708242DED0009A12F8010F0092CCE7FB
S315080021FC4FF6FF739A42E0D0019B33F81530002B4B
S3150800220CDBD0DCE706469EE6211001004FECC44EF7
S3150800221C505700085C570008012908D9F8B5056815
S3150800222C0E466B690746994203D30220F8BD022075
S3150800223C70475AB1012AF8D99342F6D9114628465D
S3150800224C4FF0FF32FFF7E0FBB0B1F8BD284614E0BB
S3150800225C314600222846FFF7D7FB0028F5D12B6913
S3150800226C5A1C05D02A79013342F001022B612A71D6
S3150800227C6B699C4211D2264638683146FFF712FB29
S3150800228C044650B10128D0D0411C08D0012ECCD917
S3150800229C6B699E42DCD30220F8BD0020F8BD0120F4
S315080022ACD3E700BF2DE9F04F0746D0F800A083B05E
S315080022BC0B780D462F2B01F10101F9D05C2BF7D0C9
S315080022CC0021B96028781F2840F2298180B21F287E
S315080022DCBE6A2FD92F282DD05C282BD00121A946D0
S315080022EC0124A6F1020800F0E9FEF8B17F2809D806
S315080022FC22281BD02A239E4A984217D012F8013F4F
S3150800230C002BF9D128F8020F19F8010F631C1F28A6
S3150800231C12D92F2810D05C280ED0B3F5807F05D0A3
S3150800232C01211C4600F0CAFE0028DFD1062003B0A6
S3150800233CBDE8F08F012300242B441A781D462F2A5A
S3150800234C03F10103F9D05C2AF7D01F288CBF4FF094
S3150800235C00094FF004094CB106EB440232F8023D71
S3150800236C202B01D02E2B07D1013CF7D100230620B8
S3150800237C338003B0BDE8F08F002220213B6A26F893
S3150800238C142003F10B0006EB440203F8011B8342ED
S3150800239CFBD1B31E4FF0000801E008F1010833F831
S315080023AC020F2028F9D02E28F7D0B8F1000F01D04B
S315080023BC49F00309134633F8022D2E2A01D0013CA5
S315080023CCF9D1002329469B463546082226461C4643
S315080023DC0B4608F1010870B320281FD02E281BD0F5
S315080023EC944220D2B0456DD07F2878D82B280AD0B5
S315080023FC2C21DFF884E104E01EF8011F002900F007
S3150800240C86808142F8D15F2049F00309396A08555C
S3150800241C013435F81800DCE7B04502D049F0030959
S3150800242CF7E794424ED30B2A00F09680B0454BD072
S3150800243C49F0030948D91D463B6A1978E52962D043
S3150800244C082A04BF4FEA8B0B5FFA8BFB0BF00C02C6
S3150800245C0C2A41D00BF0030103293DD019F0020FC9
S3150800246C0AD10BF0030BBBF1010F08BF49F0100999
S3150800247C042A08BF49F0080983F80B903846FFF779
S3150800248C83FC3B6ADB7A002854D15A073FF54FAFD9
S3150800249CBB79DB064CD53B699AF80010C3F30803E5
S315080024AC30335344D87E9A7E032942EA002202D05E
S315080024BCBA6028780AE7597D1B7D43EA012342EA6C
S315080024CC0342F5E70B2A47D04FEA8B0B5FFA8BFBD7
S315080024DCB0460B2208249CE749F00209BEE7002106
S315080024EC8DE80C0000F0EAFD9DE80C0040B121498E
S315080024FC49F00209084410F8800C002883D075E7C7
S3150800250C49F002097FE7052119703B6A98E7A0F1A3
S3150800251C4101192916D84BF0020BC0B276E7802276
S3150800252C38463B6ADA7203B0BDE8F04FFFF71EBABD
S3150800253C0520FCE604287FF4FAAE13F0040F08BF56
S3150800254C0520F4E6A0F16101192997BF2038C0B21D
S3150800255CC0B24BF0010B59E71D463B6A49F003091B
S3150800256C1A78E52A7FF472AF05221A703B6A6DE772
S3150800257C61570008D05600086D5700082DE9F84336
S3150800258C436A074601330D461AD0836A18889C1C81
S3150800259C90B1002603F5007901F1150807E0A1456D
S315080025AC0AD008F8010F34F8020B013628B10021BD
S315080025BC00F084FD0028F2D1002600232E44B375C2
S315080025CC00214FF02E080A46FE69AF7D741E14F8DA
S315080025DC013F0132202B1BD0052B08BFE523092A06
S315080025EC37D06818437297B9A3F1410EBEF1190F8B
S315080025FC0CD8092A34BF4FF0080E4FF0100E96F877
S3150800260C0CC01CEA0E0F1CBF2033DBB283750131DC
S3150800261C0B2ADCD1681827B98775337B002B08BFC2
S3150800262C284600234372F37A2B72F18B727F337F21
S3150800263C42EA012243EA02232B60727E337E43EA86
S3150800264C0223AB80F27DB37D43EA0223EB80BDE81F
S3150800265CF88368180FB980F8168080F8098001315C
S3150800266CBFE700BF2DE9F84FFF27044606683D462D
S3150800267C042006E0FF2500212046FFF7C3FA0028B0
S3150800268C59D1A16900295AD03046FEF7B9FE00285F
S3150800269C51D1E1690A78002A4CD0CB7AE52A03F0A5
S315080026AC3F03A371E6D02E2AE4D023F0200EBEF108
S315080026BC080FDFD00F2B47D1500638D523694F7B2F
S315080026CC02F0BF0563624B7BBB42D3D1CA7E8B7EBD
S315080026DC53EA0223CED1012291F800E02B480EF0E2
S315080026EC3F0E0EF1FF3E0EEB4E034FF6FF7A944665
S315080026FCD4F828900EEB830E00F10C080BE0BEF113
S3150800270CFE0FB7D89C4629F81E300EF1010E8045EF
S3150800271C2ED010F8012F8B1893F801B08B5C43EA76
S3150800272C0B23BCF1000FEAD15345F0D0A2E7AA421D
S3150800273CA0D1C8E704200023A361BDE8F88F0028C0
S3150800274CF9D10020BDE8F88F6DB90A460B3112F89D
S3150800275C016BEB0143EA550535448A4205F0FF0542
S3150800276CF5D1BD42EDD04FF0FF336362BDE8F88F6B
S3150800277C0B785B0606D5BEF1FE0F3FF67BAF002342
S3150800278C29F81E30013DEDB275E700BF5057000819
S3150800279C10B584B004AB43F8041D019018461446D2
S315080027AC0091FEF7B9FD021E0FDB0F4951F82230D6
S315080027BC0BB100201870019B8BB10020012C1870EE
S315080027CC41F8223004D004B010BD0B2004B010BD63
S315080027DC024601A96846FEF7CFFE04B010BD18469E
S315080027EC41F82230EFE700BFD40E00202DE9F04166
S315080027FC92B0019160B3002302F01F0703600446F0
S3150800280C154603A93A4601A8FEF7B6FE064618B1C0
S3150800281C304612B0BDE8F081039B5B4A079307A8C4
S3150800282C04AB019911920F93FFF73CFDA8B90F9BC6
S3150800283C93F90B30002B5BDB15F01C0F14D09DF8AD
S3150800284C223013F0110F3DD16D0746D50826DFE768
S3150800285C0926304612B0BDE8F08115F01C0F01D0E0
S3150800286C042833D00646D3E79DF82230D9062BD454
S3150800287CAA0701D5DB0725D415F0080F039D01D04F
S3150800288C47F02007EA6A0E9B226263622978D87E93
S3150800289C9A7E032942EA002223D00021A260D88B13
S315080028AC5A7F1B7F2774617442EA0022E88843EA40
S315080028BC0223A0803046E36025606161E16112B0B5
S315080028CCBDE8F0810726A3E70426A1E707A8FFF7CA
S315080028DC31FB0028C6D147F0080738070AD4039DF0
S315080028ECD0E7587D197D41EA002142EA0142D4E736
S315080028FC06268DE70022482161204FF0200E0E9BFC
S3150800290C039D59749A73DA7318740E9B59769A75D3
S3150800291CDA7518760E9B83F80BE00E9B2A78D97E0F
S3150800292C93F81A80032A48EA012825D000229A76B9
S3150800293CDA762978032904BF1A755A7501210022FB
S3150800294C0E9B1A775A779A77DA77E970B8F1000FEF
S3150800295C96D007A84146ED6AFFF75EFC002881D1A0
S3150800296C29460398FEF74CFD039D08F1FF33EB60EF
S3150800297C002885D006464BE7597D1A7D42EA012286
S3150800298C48EA0248D2E700BFDC0E00202DE9F04FDA
S3150800299C9946002385B08846C9F8003003A9144621
S315080029AC0546FEF7DBFC064628B96E7C1EB92B7C61
S315080029BCD80704D40726304605B0BDE8F08F6A69F7
S315080029CCEF68BF1AA74228BF2746002FF3D0C2F3D9
S315080029DC080305F1280A002B43D103994B89013BBF
S315080029EC13EA522349D1002A69D1A868012875D956
S315080029FC411C61D00399A8614A690238023A90428F
S31508002A0C6CD24A898C6A00FB0244002C66D05FEAB9
S31508002A1C572B1C4433D003EB0B00904288BFA2EB18
S31508002A2C030B48785B462246414602F049F80028D3
S31508002A3C42D12B7C5A0603D5E869001B834545D839
S31508002A4C4FEA4B246A69D9F80030224423443F1BC9
S31508002A5C6A61A044C9F80030ADD0C2F30803002B54
S31508002A6CBBD0C3F50074BC4228BF3C462833E918D2
S31508002A7C22464046FEF792FCE4E7A869BCE7EA69F9
S31508002A8C944214D02B7C5B060AD548780123514610
S31508002A9C02F066F880B92B7C039923F040032B745B
S31508002AAC487801232246514602F00AF820B96B6988
S31508002ABCEC61C3F30803D4E701266E747BE7A969B6
S31508002ACC28680193FEF7EEFE019B8FE708EB402082
S31508002ADC4FF400725146FEF761FCB1E702266E749C
S31508002AEC69E700BF2DE9F04F9A46002385B0894661
S31508002AFCCAF8003003A916460446FEF72FFC07460B
S31508002B0C28B9677C1FB9227C910704D40727384655
S31508002B1C05B0BDE8F08F6369F34228BFDE43002E8B
S31508002B2C00F08D8004F12802019251E0039AB2F864
S31508002B3C0AB00BF1FF3B1BEA532B0ED1002B77D1B6
S31508002B4CA06800287FD0012800F09B80421C6CD01E
S31508002B5CA368A061039A03B9A060237C5B0657D4CB
S31508002B6CA1695369A1F10208023B984580F0898056
S31508002B7C5389916A08FB0311002900F08280750AB3
S31508002B8C0BEB010838D00BEB0501994288BFA3EB78
S31508002B9C0B0550782B464246494601F0E1FF0028C2
S31508002BAC43D1E169A1EB08018D425ED86D026369D8
S31508002BBCE2682B449A4238BF1A461146DAF80020C6
S31508002BCC761B2A446361E160A944CAF8002035D013
S31508002BDCC3F308000028A9D0C0F50075B54228BF74
S31508002BEC3546283020442A464946FEF7D7FB237C2F
S31508002BFC43F040032374DAE7E3696069984502D029
S31508002C0CE368984227D3C4F81C80C0F30800E3E7AE
S31508002C1C50780123E269019901F0A2FF28B9237CB7
S31508002C2C039A23F0400323749AE7012767746EE727
S31508002C3CA1692046FEF77CFF002884D1227C42F04D
S31508002C4C2002227463E759462046FEF771FF0028D6
S31508002C5C7FF479AFF2E7507801234246019901F0E7
S31508002C6C2FFF0028E1D16069CDE709EB41214FF42C
S31508002C7C00720198FEF792FB237C23F04003237421
S31508002C8C94E70227677442E770B50A2982B00E46A4
S31508002C9C05461AD06C68002C08DB2B1901343C2C21
S31508002CAC1E7305DCAB686C600133AB6002B070BD9B
S31508002CBC01AB224605F10C012868FFF713FF019BAF
S31508002CCC1C1B18BF4FF0FF34ECE70D21FFF7DCFF98
S31508002CDCE0E700BFF0B583B001A90446FEF73EFB5A
S31508002CEC002844D1237C9A0641D55B060DD5019A5A
S31508002CFC0123507804F12801E26901F031FF00281C
S31508002D0C37D1237C23F040032374216A0198FEF7FC
S31508002D1C77FB60BB636ADA7A42F02002DA72A26841
S31508002D2C2168C2F30720D8769A760978032922D027
S31508002D3C0021482061270126E268019D4FEA122EE0
S31508002D4C1A7783F81DE04FEA124E120E587683F85E
S31508002D5C1EE0DA779975D9759974D9741F76284651
S31508002D6CEE70FEF76BFB237C23F02003237403B071
S31508002D7CF0BD0120FBE7120C110A1A755975D7E735
S31508002D8C10B582B00446FFF7A5FF08B102B010BD16
S31508002D9C01A92046FEF7E2FA0028F7D1206002B016
S31508002DAC10BD00BF2DE9F04182B00E4601A90446BC
S31508002DBCFEF7D4FA0746002842D1677C002F3FD18C
S31508002DCCE368B34204D2227C12F0020F08BF1E46F7
S31508002DDC002263696261002E32D0019AB2F80A8029
S31508002DEC4FEA48283BB1013B721EB3FBF8F1B2FB24
S31508002DFCF8F28A4259D2A568002D62D0A5611DBB8E
S31508002E0C6369C3F30802002A66D0E269954263D067
S31508002E1C237C5B063AD404F12806019B3146587884
S31508002E2C2A46012301F04CFE002838D16369E26872
S31508002E3CE561934204D9227CE36042F020032374B3
S31508002E4C384602B0BDE8F081464514D847E020461E
S31508002E5CFEF76EFE0546002840D06A1C1FD0012DD1
S31508002E6C20D9019B5B699D421CD26369B0454344DA
S31508002E7CA561636134D2237CA6EB0806980729461C
S31508002E8CE5D42068FEF70EFD0546E6E7019B04F13E
S31508002E9C280658783146012301F062FE60B10127F5
S31508002EAC6774CDE702276774CAE7C8F100021340B6
S31508002EBC6361F61AA569A2E7237C23F04003237401
S31508002ECCABE729462046FEF733FE01280546E9D02E
S31508002EDC431CE4D0A06091E7E268AAE7464663691A
S31508002EEC3344C6F30802636172B10199023D4A691B
S31508002EFC023A9542D6D24A89896A05FB0215002DF3
S31508002F0CD0D005EB56257CE715467AE730B591B057
S31508002F1C01900D46002205A901A8FEF72DFB0446D3
S31508002F2C10B1204611B030BD0F4A02AB019905A865
S31508002F3C0F920D93FFF7B6F904460028F1D10D9BB5
S31508002F4C93F90B30002B0ADB002DEAD00B9BA875E6
S31508002F5C002BE6D0294605A8FFF710FBE1E7062467
S31508002F6C204611B030BD00BFDC0E002030B59DB038
S31508002F7C0190022202A901A8FEF7FEFA029B06930B
S31508002F8C08B11DB030BD254A03AB06A801991092AD
S31508002F9C0E93FFF787F90028F3D10E9B93F90B30A4
S31508002FAC002B05DB9DF81E30DA0703D50720E8E76A
S31508002FBC0620E6E7029D0D9A2978D07E947E032991
S31508002FCC44EA00241BD0DB0609D406A8FEF7B4FE97
S31508002FDC0028D6D1D4B90298FEF730FAD1E711A851
S31508002FEC002111951394FEF7C1FC0028C9D111A82C
S31508002FFCFFF738FB0028D9D00428E6D0C1E7517D65
S3150800300C127D42EA012244EA0244DCE702462146E2
S3150800301C06A8FFF701F90028B3D1DCE7DC0E00207F
S3150800302C2DE9F041804617460546002482B04E1E0F
S3150800303CA64212DD01AB012269463846FFF7A6FC0B
S3150800304C019B012B09D19DF800300D2BF0D00A2BD2
S3150800305C05F8013B04F10104EAD100239C4214BF94
S3150800306C404618462B7002B0BDE8F08110B50446F0
S3150800307C00230846217894B0019002930393D1B1AA
S3150800308C01A8FFF701FE14F8011F0029F8D1029ACE
S3150800309C002A0CDB01986B4604A9FFF723FD30B90F
S315080030AC029A009B9A4202D1039814B010BD4FF0B5
S315080030BCFF3014B010BD0A46EDE700BF7F2811D9C2
S315080030CC89B910B40E4AC72303E0802914D032F804
S315080030DC023F98428CB201F10101F6D104F180004D
S315080030EC10BC80B27047FF2804D8054B803833F8DB
S315080030FC1000704700207047002010BCF2E700BF94
S3150800310C74570008274AB0F5805F274B41F67D5166
S3150800311C3CBF13466121043399B1884211D370B46C
S3150800312C33F8022C1E46D4B26518A8424FEA12226E
S3150800313C08DB04337AB133F8041C09B18842EFD2A0
S3150800314C70BC7047082AFBD8DFE802F00F13191C6D
S3150800315C1F2225280B0006EB440336F814100433FB
S3150800316CEBE7A0F5E35080B2EAE7411A33F8110011
S3150800317CE6E7411A01F00103C01A80B2E0E71038FD
S3150800318C80B2DDE7203880B2DAE7303880B2D7E78C
S3150800319C1A3880B2D4E7083080B2D1E7503880B2FA
S315080031ACCEE700BF74580008685A00080022054B81
S315080031BC1A709A6483F84220A3F844209A705A70BD
S315080031CC704700BFDC100020024B1878003018BF7F
S315080031DC01207047DC1000200022024B83F84220A5
S315080031EC704700BFDC100020F8B50578FF2D41D0DC
S315080031FCB24C2378012B00D0F8BDC93D0646352DB7
S3150800320C00F24081DFE815F010013E013E018F0007
S3150800321C3E013E0197007C009F00A6003E013E0140
S3150800322C3E013E013E013E013E013E013E013E018C
S3150800323C3E013E013E013E013E013E013E013E017C
S3150800324C3E013E013E013E013E013E013E013E016C
S3150800325C3E013E013E013E013E013E01B500D10054
S3150800326CDE0027013E013E013E012F013E01F20020
S3150800327CFA000701FDF708FDE8B9FE211022022322
S3150800328C8E4CE1702271A4F8443094F84230012B2C
S3150800329C09D0B4F84410012384F842308848BDE8B4
S315080032ACF840FDF75FBCFE2210230221E270237161
S315080032BCA4F84410EFE70023102201267F4C637014
S315080032CC63712271E5702670FDF76CFCA071FDF731
S315080032DC5BFCE071FDF758FC0823D8402072667237
S315080032ECA672A4F84430FDF7CBF994F84230012BBA
S315080032FCD9D0B4F9441000297FF77EAF89B2CAE752
S3150800330CFDF750FC73780138984253DDFF220123F0
S3150800331CE270A4F844307178002940F0C080FDF7BB
S3150800332CB9F90028E1D1FE2131220223E17022717C
S3150800333CA4F84430A9E7FCF709FFFF220123E27041
S3150800334CA4F84430A1E74168A06CFDF79DF9002864
S3150800335CF3D1E8E70025FF232571E3706571FDF7C6
S3150800336C21FC0723A071E57125726572A4F8443017
S3150800337C8BE7FF23E3704768A66C002F00F09B8051
S3150800338C0025374416F8013B1D44FDF711FCBE42D7
S3150800339CEDB2F7D1002301210822C4F80750217198
S315080033AC6371A371A4F844206FE7FDF7FBFB7378F0
S315080033BC98426FDCFE2122220223E1702271A4F8C6
S315080033CC443062E7FDF7EEFB72789042F2DDA16CB1
S315080033DC3C48FCF7DBFEFF23E3707278A36C1344BE
S315080033ECA36473780133A4F844307EE7FE210022E7
S315080033FC0223E1702271A4F8443046E70023FF202B
S3150800340C06216278E0702371A371E3712372A4F824
S3150800341C4410627139E70023FF210122237063707F
S3150800342CE170A4F8442030E7A56CFDF7BBFB721CD1
S3150800343C411E2846FDF726F900283FF474AFFF23F2
S3150800344CE370FDF7AFFB0122A36C01380344A364B8
S3150800345CA4F8442019E7FF230122E3704368A4F873
S3150800346C4420A36411E70023FF2507200821164AE8
S3150800347CE57023716371A371C4F80700A4F84410AE
S3150800348CA26402E7FE2120220223E1702271A4F82D
S3150800349C4430FAE671680B48A164727899E7B21C55
S315080034ACA06CFDF7EFF800283FF43DAF7278A36CDB
S315080034BC1344A36419E73D466CE700BFDC100020F3
S315080034CCDF100020E0100020245B000830B5174CF4
S315080034DC83B02378054643B1012D4FF48051144827
S315080034EC1FD000F03BF903B030BD0121102000F0CD
S315080034FC39F94FF480501423032202A921F8040D3C
S3150800350C00F1804000F580308DF807308DF80620E4
S3150800351C00F0C0F80123012D23704FF480510448A4
S3150800352CDFD100F01DF903B030BD00BF2811002013
S3150800353C0010014008B50121034800F009F910B143
S3150800354C00F0A2F8012008BD00080140642000F034
S3150800355C6FB800BF00F072B800B5C7B00021684656
S3150800356C4FF48C7201F042FF69460948FFF7CEFC0E
S3150800357C50B9009828B19DF8080080F01000C0F3E7
S3150800358C001047B05DF804FB002047B05DF804FB5B
S3150800359C3C5B0008004870473C5B0008002310B5EC
S315080035AC064C0A222046064984F82832FFF71EF9EB
S315080035BC10B9012384F8283210BD00BF2C11002045
S315080035CC2C5B000808B5084890F82832012B04D063
S315080035DCBDE808400548FFF7C9BCFFF7D1FBBDE8B5
S315080035EC08400248FFF7C2BC2C1100203C5B0008BF
S315080035FC034890F82832012B00D07047FFF7C0BB60
S3150800360C2C11002010B5094C94F82832012B00D047
S3150800361C10BD2146FFF72AFD0028F9DA002384F8A5
S3150800362C28322046BDE81040FFF7AABB2C11002013
S3150800363C014B1880704700BF5813002010B5FDF7D2
S3150800364C5BF80D4C236898420ED30C4B1A7862B172
S3150800365C002220210A481A7000F082F8FDF74CF86F
S3150800366C084B1B881844206010BD012220210448F1
S3150800367C1A7000F073F8F1E75C1300205A13002057
S3150800368C00080140581300202021014800F068B8B2
S3150800369C000801402DE9F041CD78EB0648BF8B7840
S315080036AC098805F00F0E48BF4EEA030E11F0FF0FFE
S315080036BC20D0002301274FF00F08066802E00133DB
S315080036CC082B16D007FA03F232EA0104F7D19C004C
S315080036DC08FA04FC26EA0C060EFA04F4282D46EA27
S315080036EC040632D0482D03F1010308BF0261082BEA
S315080036FCE8D10660FF2924D90022082301274FF0B8
S3150800370C0F08466804E00133102B02F1040217D0A7
S3150800371C07FA03F434EA010CF5D108FA02FC26EA96
S3150800372C0C06282D0EFA02FC4CEA06060BD0482D80
S3150800373C03F1010308BF0461102B02F10402E7D15F
S3150800374C4660BDE8F0814461DDE74261B7E700BF3A
S3150800375C8368194214BF0120002070470161704725
S3150800376C41617047044A936919B923EA00009061CC
S3150800377C704718439061704700100240044AD36999
S3150800378C19B923EA0000D06170471843D061704715
S3150800379C001002404A880B8830B48C881343CA88B8
S315080037AC23430C8913434A898D8923431343CC89B4
S315080037BC02882B43234302F4415213439BB20380E2
S315080037CC838B0A8A23F400631B041B0C838330BC8B
S315080037DC02827047038829B923F040031B041B0C8B
S315080037EC038070479BB243F040030380704700BFC9
S315080037FC81817047808980B2704700BF038829B9D8
S3150800380C23F400531B041B0C038070479BB243F430
S3150800381C00530380704700BF0389194214BF012067
S3150800382C0020704708B538B1064B1B681B689847CB
S3150800383C054B18680A3008BD0122034B1B681A820F
S3150800384C08BD00BF9C130020A013002008B538B192
S3150800385C064B1B689B689847054B18680C3008BDC7
S3150800386C0122034B1B681A8208BD00BF9C1300205B
S3150800387CA013002008B5002833D000211E4B1F4882
S3150800388C1A680180137813F07F0316D0012B27D002
S3150800389C022B24D1527902F00F039B0003F18043CB
S315080038AC03F5B84312061B6820D403F44053B3F54A
S315080038BC805F0ED1012303700BE0527A93064CBF3E
S315080038CC0223037851064CBF43F0010323F001038E
S315080038DC03700B4B1B681B699847084808BD0846BC
S315080038EC08BD0222044B1B681A8208BD03F030037C
S315080038FC102BEED1DEE700BFA013002070130020BA
S3150800390C9C1300202DE9F041244F3D682C8A2CB9D4
S3150800391C2E7A042E2BD0AB8A042604E0AB8A9C4262
S3150800392C8CBF022604269C4228BF1C46AB6920463F
S3150800393C98478046002000F01DFE22460146404668
S3150800394C00F0EAFC2146002000F0B2FD30204FF4CE
S3150800395C40522B8A698A1B1B2B820C44104B11492B
S3150800396C6C8208803D681A802E72BDE8F0810E4B79
S3150800397C1A78012A06D0102207260A4B1A802E72AC
S3150800398CBDE8F08130270949094A0968054889B212
S3150800399C0A44520014601C700780E5E7A013002047
S315080039ACA6130020A813002060130020505C0040CA
S315080039BC023000200B4B0C4A1B685178DA7891427E
S315080039CC01D20220704799780029FAD110B59C8843
S315080039DC0CB1022010BD05499A720B685B689847B2
S315080039EC204610BDA0130020A00000209C13002028
S315080039FC10B5114A114C1268236882B0D9785879D7
S31508003A0C9369984723689A7A12B9022002B010BDB6
S31508003A1C0028FAD11A79002AF7D19B78002BF4D111
S31508003A2C074B01901B68DB689847236801985979FE
S31508003A3CDA78D9721A73E9E778130020A0130020F4
S31508003A4C9C13002038B5344B1B68187810F07F008F
S31508003A5C03D0022806D0022038BD5A7A22F020025A
S31508003A6C5A7238BD5A88002AF6D11A79002AF3D127
S31508003A7C58792A4D44B220F08000810001F1804229
S31508003A8C02F5B84212682D78002CB4BF02F0300249
S31508003A9C02F44052A842DED2002ADCD09B7A002BD4
S31508003AACD9D0002C0FDB01F1804404F5B844236807
S31508003ABC03F44053B3F5805F17D0194B1B685B6949
S31508003ACC9847002038BD01F1804101F5B8410B68D3
S31508003ADC03F03003102BF0D1C4B2204600F0D6FC0C
S31508003AEC2046302100F052FCE7E790B90D4B93F8CD
S31508003AFC2C1000F0EBFC236823F4804323F07003AE
S31508003B0C9BB283F4405343F4004343F08003236091
S31508003B1CD3E700F0A9FCEEE7A0130020A0000020D4
S31508003B2C9C1300207000002038B5234B234D1968D0
S31508003B3C2D784B795CB223F08003980000F1804213
S31508003B4C02F5B8421268002CB4BF02F0300202F437
S31508003B5C4052AB4201D3022038BD4B88002BFAD118
S31508003B6C002AF8D08B7A002BF5D000F1804000F5AE
S31508003B7CB840002C036811DB23F4804323F0700350
S31508003B8C9BB283F4805343F4004343F080030360F1
S31508003B9C0B4B1B689B699847002038BD23F4E04300
S31508003BAC23F040039BB283F0100343F4004343F025
S31508003BBC80030360ECE700BFA0130020A0000020E0
S31508003BCC9C130020054B1B685A8A10B108681044D0
S31508003BDC704789888A1A1A82704700BFA01300207A
S31508003BEC10B50C4B002093F82C1000F06FFC0A4B08
S31508003BFC1B68187A082806D14FF4805410220749F6
S31508003C0C074B0C801A80A0F10900B0FA80F0400925
S31508003C1C10BD00BF70000020A0130020A6130020C2
S31508003C2CA813002070B5A94EA94B34681A68237AD4
S31508003C3C82B0092B3CD0A74B92B213445B001D886B
S31508003C4C6D0005F1804505F5C0452B7823706B781A
S31508003C5C6370A88800F0B2FC60802889346800F08C
S31508003C6CADFC0122A080AB893468E380227223B3B1
S31508003C7C6078062800F0838000283AD161880029EC
S31508003C8C00F09380944D2B681B699847032800F025
S31508003C9CE3804FF6FF723468238A934200F08380E0
S31508003CAC022836D108232372FFF79AFF02B070BD9B
S31508003CBC0122E3882272002BDAD12378657813F077
S31508003CCC7F0336D0012B00F0BA80022B00F0DD8082
S31508003CDC814B28461B685B699847032800F00E81C0
S31508003CEC346800283ED008232372FFF779FF02B008
S31508003CFC70BD08286BD123785B06C3D1774B00209F
S31508003D0CA361608298474FF6FF723468238A934200
S31508003D1C49D0002BC6D094F90020002A7ADB03215F
S31508003D2C4FF440526E4B21721A80FFF759FF02B0BE
S31508003D3C70BD092D00F0C480052D00F09480032D6C
S31508003D4C00F0AC80012DC3D1E378012BC0D1A38838
S31508003D5C002BBDD1637A9B06BAD5FFF773FE0028F4
S31508003D6CB6D1346800253020594A5E4B12685E4934
S31508003D7C92B213445B001D6006230880B4E72378CF
S31508003D8C5D067FF47FAFA378534D012B00F09B8023
S31508003D9C022B65D0032B7FF476AF2B685B6A002B5E
S31508003DACADD106206FE709239EE7636823F47F43AA
S31508003DBCB3F5003F7FF466AF207810F07F0040F033
S31508003DCCA080A388002B7FF45DAF484B97E70A28A1
S31508003DDC7FF458AF237803F07F03012B7FF452AF9F
S31508003DECA37A002B3FF44EAF618800297FF44AAFC3
S31508003DFC6368394D23F47F43B3F5803F7FF443AFB3
S31508003E0C2B6860799B699847002840F0B68034681F
S31508003E1C374B74E7E288019201998B4215D89A427E
S31508003E2C75D92D4A126892F82C108AB29A4273D90F
S31508003E3C0021304B1970A282FFF764FD55E70B2D54
S31508003E4C7FF446AFFFF7D4FD89E7234B019A1B682D
S31508003E5C228293F82C20EEE7092233681A7244E77B
S31508003E6C2B681B6A9BE794F90330002BFFF63BAFD4
S31508003E7CA378002B7FF437AFA388002B7FF433AFDE
S31508003E8CA37A002B3FF46EAF2DE7012D3FF465AFF7
S31508003E9C032D7FF41DAFFFF747FE60E7E378012B90
S31508003EAC7FF416AFA388002B7FF412AF637A124AFD
S31508003EBC43F0200312686372D3699847346851E754
S31508003ECCFFF778FD4BE72B68DB6968E7A013002042
S31508003EDC505C00400430002078130020313800086C
S31508003EECA613002002300020A813002081380008F1
S31508003EFC59380008601300209C13002034680923E5
S31508003F0CF2E601282CD0022810D00020BAE61C4B69
S31508003F1C1B6893F82C208EE793FBF1F001FB10330A
S31508003F2C002B88D10121174B197084E7607900F0B2
S31508003F3C0F029300010603F18043134903F5B843B6
S31508003F4C1B6809784CBF03F0300303F440538A42CC
S31508003F5CDBD210F07000D8D1002B7FF436AF91E687
S31508003F6C074D60792B689B69984730B93468A37AF2
S31508003F7C002B7FF42AAF607885E63368587882E69A
S31508003F8C7813002060130020A0000020F8B5334DEC
S31508003F9C2C68237A022B07D0042B05D0032B09D0C7
S31508003FAC052B07D0072B36D008232372BDE8F8401B
S31508003FBCFFF716BEA369228ABBB1002A32D0A68A9D
S31508003FCC964228BF164630469847228A638A921B21
S31508003FDC3344074622826382002000F0DBFA32461D
S31508003FEC0146384600F0ACF9228A02B300214FF498
S31508003FFC405230261A4B08461A8000F059FA238A82
S3150800400CA18A184899422A68068022D91BB3052327
S3150800401C14461372C9E7144B1B68DB6898472C685F
S3150800402C0823C2E7A38A33B903232372BDE7A38AFD
S3150800403C2C68002BF8D00B480623002630250B4A93
S3150800404C237211680A4A89B20A445200166005801E
S3150800405CABE71446E8E71446EEE700BFA0130020CA
S3150800406CA6130020A813002078130020505C0040EB
S3150800407C02300020F8B5234C23681A7A022A17D086
S3150800408C042A15D0062A05D008221A72BDE8F8406B
S3150800409CFFF7A6BD5A78052A13D01B4B1B689B68DD
S315080040AC9847082223681A72BDE8F840FFF798BDAE
S315080040BCFFF728FC23681A7A1A72BDE8F840FFF74E
S315080040CC8FBD1A7812F07F02E7D1104993F803E0F6
S315080040DC0D7875B140F60F7748F280060C490B68D7
S315080040EC42EA06003B4001320343954241F8043B41
S315080040FCF5D10849084A4EF080030B6013681B6A11
S3150800410C9847CAE7A013002078130020A0000020C7
S3150800411C005C00404C5C00409C130020F0B40C4B37
S3150800412C1D787DB1002240F60F7748F280060949C2
S3150800413C0B6842EA06043B4001322343954241F898
S3150800414C043BF5D1044B40F080001860F0BC704776
S3150800415CA0000020005C00404C5C0040704700BF8B
S3150800416C70B40226064A074D074C084B08490948FD
S3150800417C167223602A601B68086070BC184700BF5B
S3150800418C80130020A0130020781300207000002054
S3150800419C9C130020CC00002000232DE9F047564E36
S315080041AC84B0DFF86C91DFF86C81544FADF80E30A3
S315080041BCD9F80030524C99B21B04524D524A3180F0
S315080041CC40F18E80338803F00F03990001F180418A
S315080041DC01F5B84188F80030002B30D14BF6BF7A80
S315080041EC23689BB22B802B8803F0300313802B8813
S315080041FC03F440532B80236803EA0A0383F4005321
S3150800420C83F0200343F4004343F080032360338890
S3150800421CD8063CD523689BB2ADF80E30BDF80E30E7
S3150800422C190560D4BDF80E301B04C1D540F68F7144
S3150800423C236801920B402360FFF7A8FE2FE00A685B
S3150800424C92B2ADF80E20BDF80E20100414D4BDF8A9
S3150800425C0E301A06ACD548F60F7098F80020930065
S3150800426C03F1804303F5B8431968013A014057F83E
S3150800427C2220196090479BE740F68F740A682348FA
S3150800428C2240013B50F823300A609847DFE748F68E
S3150800429C0F71236801920B402360FFF7EBFE23682E
S315080042AC298803EA0A0A019A2B8811F4805F18BF39
S315080042BC8AF4805A9E04138848BF8AF4005ADD068D
S315080042CC138848BF8AF0100A9C0648BF8AF0200A51
S315080042DC4AF4004A4AF0800A094A1FFA8AF313601C
S315080042EC04B0BDE8F08740F68F71236801920B4045
S315080042FC2360FFF797FCD2E7AA13002020000020C2
S3150800430C005C0040A6130020A81300203C000020E7
S3150800431C445C00407C130020013252100ED000235E
S3150800432C10B401F1005101F54051490030F8024B27
S3150800433C21F8234001339A42F8D110BC704700BFCC
S3150800434C01F10051013201F5405152104FEA410179
S3150800435C05D051F8043B013A20F8023BF9D17047D5
S3150800436C4FF6F873014A034013607047505C0040DF
S3150800437C800000F1804000F5B840036823F4EC4354
S3150800438C23F07003194389B201607047800000F16D
S3150800439C804000F5B8400368CA0623F4E04323F0CE
S315080043AC40039BB248BF83F010038A0648BF83F0CC
S315080043BC200343F4004343F080030360704700BFB7
S315080043CC800000F1804000F5B8400368CA0423F465
S315080043DC804323F070039BB248BF83F480538A044E
S315080043EC48BF83F4005343F4004343F0800303604F
S315080043FC704700BF800000F1804000F5B8400368A4
S3150800440C23F4E04323F040039BB283F0300343F4D8
S3150800441C004343F080030360704700BF800000F13F
S3150800442C804000F5B840036823F4804323F07003FA
S3150800443C9BB283F4405343F4004343F08003036078
S3150800444C704700BF40F60F63800000F1804000F50E
S3150800445CB8400268134043F4004343F080030360FA
S3150800446C704700BFFFF7EEBF800000F1804000F5F3
S3150800447CB84003685B0408D540F60F72036813400E
S3150800448C43F4404343F0800303607047800000F117
S3150800449C804000F5B84003685B0608D540F60F72F5
S315080044AC0368134043F4004343F0C00303607047AA
S315080044BC044A054B126892B202EBC00003445B0037
S315080044CC19607047505C0040023000200E4A0F4BB2
S315080044DC12683E2992B202EBC00003444FEA43032A
S315080044EC0AD94A09C80604BF02F1FF3292B29202EF
S315080044FC42F400421A6070474A08C90748BF01329D
S3150800450C92021A60704700BF505C004006300020CB
S3150800451C064B49081B6849009BB203EBC00000F127
S3150800452C005000F54050400001607047505C004058
S3150800453CFFF7EEBF054A064B1268490892B202EB22
S3150800454CC002134449005B0019607047505C004078
S3150800455C04300020FFF7EEBF054B1B689BB203EB3C
S3150800456CC00000F1005000F540504000008870472C
S3150800457C505C0040FFF7F0BF044A054B126892B234
S3150800458C02EBC00003445B0018887047505C00407F
S3150800459C04300020FFF7F0BF054A064B126892B2AA
S315080045AC02EBC00003445B001868C0F309007047AF
S315080045BC505C004006300020FFF7EEBFC3B2000A7D
S315080045CC40EA0320704700BF00204FF4064310B49E
S315080045DC0349044C044A20600B8010BC13607047D6
S315080045ECA4130020445C0040405C004070B500F009
S315080045FC7F0528460E46FFF7DFFF04462846FFF7D9
S3150800460CC9FF224601463046FFF79AFE204670BD82
S3150800461C014608B50648FFF7EBF801210448FFF7F1
S3150800462CFBF80028F9D00248FFF7E4F8C0B208BD39
S3150800463C0038004010B5FCF75FF800F5FA7403E093
S3150800464CFCF75AF8844206D9FF20FFF7E1FFFF284A
S3150800465CF6D1012010BD002010BD00BF10B50421F5
S3150800466C0A48FFF77DF8FF20FFF7D2FFFFF7E2FFB6
S3150800467C10B10124204610BD044604210348FFF757
S3150800468C6DF8FF20FFF7C4FF204610BD001401404B
S3150800469C38B50D46010604460BD404212248FFF70B
S315080046AC5DF8FF20FFF7B4FFFFF7D8FF58B9FF20D6
S315080046BC38BD00213720FFF7EBFF012800D938BD9C
S315080046CC04F07F04E9E744F04000FFF7A1FF280E49
S315080046DCFFF79EFFC5F30740FFF79AFFC5F30720C0
S315080046ECFFF796FFE8B2FFF793FF2CB1082C12D10F
S315080046FC8720FFF78DFF02E09520FFF789FF0A2434
S3150800470CFF20FFF785FF020604F1FF33D7D513F018
S3150800471CFF04F5D138BD0120FFF77AFF0C2CEED13A
S3150800472CFF20FFF775FFEAE70014014070B5044651
S3150800473C0D46FBF7E1FF00F1640603E0FBF7DCFF2F
S3150800474C86421DD9FF20FFF763FFFF28F6D0FE2807
S3150800475C16D10234FF20FFF75BFF04F8020CFF208A
S3150800476CFFF756FF023D04F8010C04F10204F1D1DF
S3150800477CFF20FFF74DFFFF20FFF74AFF012070BD12
S3150800478C002070BD38B505460C46FFF753FF00B937
S3150800479C38BD2046FFF73CFFFD2C1ED0AC1C05F29D
S315080047AC022514F8020CFFF733FF023414F8030C35
S315080047BCFFF72EFFAC42F4D1FF20FFF729FFFF20AD
S315080047CCFFF726FFFF20FFF723FF00F01F00A0F1DD
S315080047DC0500B0FA80F0400938BD0120D8E700BFC3
S315080047EC002840F0C1802DE9F047AB4E88B03478EC
S315080047FC14F0020404D03078C0B208B0BDE8F087D3
S3150800480C042703254FF0100A01212020FEF7AAFFE2
S3150800481C01210820FEF7A6FF01214FF48040FEF780
S3150800482CADFF0DEB07019D488DF80650ADF80470E9
S3150800483C8DF807A0FEF72EFF39469848FEF78EFF2F
S3150800484C4FF4204218230DEB070195488DF80650B6
S3150800485CADF804208DF80730FEF71CFF4FF48042A4
S3150800486C48230DEB07018E48ADF804208DF8073068
S3150800487CFEF710FF4FF482704FF4007138220723AD
S3150800488C4FF400490DF10C08ADF80E00ADF81610F2
S3150800489C84484146ADF81820ADF81C30ADF80C40EC
S315080048ACADF81040ADF81240ADF81440ADF81A400A
S315080048BCFEF770FF21467B48FEF7A0FF01217948D9
S315080048CCFEF788FF39467548FEF748FF02A9744873
S315080048DC8DF80A508DF80BA0ADF80890FEF7DAFEA5
S315080048EC49466F48FEF73AFF0A256E4C02212046C8
S315080048FCFEF792FF0028F9D0FF212046FEF778FF35
S3150800490C01212046FEF788FF0028F9D0013DEDD19C
S3150800491C4FF400400322182302A9ADF8080060489A
S3150800492C8DF80A208DF80B30FEF7B4FE04215B488F
S3150800493CFEF716FF29462846FFF7AAFE0128044665
S3150800494C14D00022584B042154481A60FEF706FF6F
S3150800495CFF20FFF75DFE337843F0010333703078A0
S3150800496CC0B208B0BDE8F08701207047FBF7C4FE5B
S3150800497C4FF4D57100F57A770820FFF789FE0128E0
S3150800498C34D102AC2546FF20FFF742FE05F8010B91
S3150800499CA845F8D19DF80A30012BD2D19DF80B30D9
S315080049ACAA2BCED105E04FF08041A920FFF770FE67
S315080049BC18B1FBF7A1FE8742F5D8FBF79DFE874297
S315080049CCBFD900213A20FFF763FE0028B9D1FF2092
S315080049DCFFF71EFE04F8010BAC42F8D19DF808301F
S315080049EC13F0400F14BF0C2504251DE02946A920F9
S315080049FCFFF74EFE012896BFA9240125022504E0DF
S31508004A0C00212046FFF744FE18B1FBF775FE8742D6
S31508004A1CF6D8FBF771FE874293D94FF40071102034
S31508004A2CFFF736FE00288CD11F4A04211B48156057
S31508004A3CFEF794FEFF20FFF7EBFD002133781948AB
S31508004A4C03F0FE030C4633704FF48277FEF7C2FE72
S31508004A5C4FF400750822072341461248ADF8182072
S31508004A6CADF81C30ADF80C40ADF81040ADF812405E
S31508004A7CADF81440ADF81A40ADF80E70ADF81650F6
S31508004A8CFEF788FE21460748FEF7B8FE01210548C1
S31508004A9CFEF7A0FEAFE600BF01000020001401409F
S31508004AAC000C0140003800406413002018B9034B71
S31508004ABC1878C0B270470120704700BF010000206B
S31508004ACC10B582B018B10424204602B010BD002BD4
S31508004ADCF9D00C461F490978C80701D50324F3E712
S31508004AEC1D4901930968090758BF5202012B114643
S31508004AFC20D01220FFF7CCFD019B58B101240421CC
S31508004B0C1648FEF72BFEFF20FFF782FDDCE7019B1C
S31508004B1C013B1DD020464FF400710193FFF706FEAA
S31508004B2C04F500740028F2D1012400210C20FFF7AB
S31508004B3CAFFDE4E71120FFF7ABFD0028DED12046D8
S31508004B4C4FF40071FFF7F2FDB0FA80F46409D6E76A
S31508004B5C1C46EAE7010000206413002000140140FB
S31508004B6C10B582B018B10424204602B010BD002B33
S31508004B7CF9D00C462A490878C00701D50324F3E76F
S31508004B8C0978490701D50224EEE72649096808077A
S31508004B9C58BF5202012B35D011F0060F29D11146F8
S31508004BAC19200093FFF774FD009B50B101240421D2
S31508004BBC1D48FEF7D3FDFF20FFF72AFDD4E7013B7E
S31508004BCC09D02046FC210093FFF7DCFD04F50074A0
S31508004BDC009B0028F3D10093FFF72CFD009B0028BF
S31508004BECE4D01C1C4FF0FD0018BF0124FFF710FD84
S31508004BFCDDE71946972001920093FFF749FD019AC4
S31508004C0C009BCCE711461820FFF742FD0028CDD1B2
S31508004C1C2046FE21FFF7B6FDB0FA80F46409C6E714
S31508004C2C01000020641300200014014070B584B004
S31508004C3C18B10424204604B070BD844B1B78D807E1
S31508004C4C03D50324204604B070BD15460E2900F280
S31508004C5CA480DFE801F05F65A229A2A2A2A2A2A203
S31508004C6C5A4C9A1808007A4B1B685B0700F1BB80F4
S31508004C7C012404217748FEF771FDFF20FFF7C8FCD5
S31508004C8C204604B070BD00213A20FFF701FD00282C
S31508004C9CEED16C1E0335FF20FFF7BAFC04F8010FA2
S31508004CACAC42F8D10024E4E7694C236813F00401FC
S31508004CBC75D000218D20FFF7EBFC0028D8D1FF20FA
S31508004CCCFFF7A6FC10216846FFF730FD0028CFD069
S31508004CDC3024FF20013CFFF79BFC14F0FF04F8D1AD
S31508004CEC10239DF80A20120993402B60C1E7002176
S31508004CFC0920FFF7CDFC0028BAD128461021FFF76A
S31508004D0C15FDB0FA80F46409B3E7514B00241B680F
S31508004D1C1370AEE7FFF7A2FCB0FA80F46409A8E7B3
S31508004D2C00210920FFF7B4FC04460028A0D1102165
S31508004D3C6846FFF7FBFC00289AD09DF800309B09C3
S31508004D4C012B62D09DF805309DF80A609DF8090084
S31508004D5C03F00F039DF807209DF8061003EBD613F6
S31508004D6C40009DF80860023300F0060092008902A4
S31508004D7C034402EB961201F44061DBB20A44093B88
S31508004D8C013202FA03F32B6073E700210A20FFF7BE
S31508004D9C7FFC00287FF46CAFAFE7042469E7092091
S31508004DACFFF776FC064600287FF462AF10216846AA
S31508004DBCFFF7BCFC00283FF45BAF246814F0020430
S31508004DCC33D09DF80A309DF80B105B009DF80D202A
S31508004DDC03F07E0303EBD11392090133013A934096
S31508004DEC34462B6045E700218D20FFF751FC00283F
S31508004DFC7FF43EAFFF20FFF70BFC28464021FFF758
S31508004E0C95FCB0FA80F4640933E79DF807309DF8F1
S31508004E1C08101B049DF8092003F47C13013302EBDC
S31508004E2C012213449B022B6023E79DF80B109DF877
S31508004E3C0A30CA0002F01802C3F3840302EB5112BB
S31508004E4C013302FB03332B6013E700BF010000207C
S31508004E5C641300200014014030B400244FF41F05DD
S31508004E6C3A4B3B49186882B040F001001860586804
S31508004E7C1A4601405960196821F0847121F4803171
S31508004E8C1960196821F480211960596821F4FE010A
S31508004E9C59609D6000940194196841F48031196039
S31508004EAC03E0009BB3F5A06F09D0136803F4003335
S31508004EBC0193009B01330093019B002BF1D0234BEC
S31508004ECC1B6813F4003318BF01230193019B012BB4
S31508004EDC06D04FF000621F4B9A6002B030BC704788
S31508004EEC1D491A4B08681A4640F0100008600868F5
S31508004EFC20F003000860086840F002000860596852
S31508004F0C596059685960596841F480615960596803
S31508004F1C21F47C115960596841F4E81159601968F3
S31508004F2C41F08071196013689B01FCD553680749D9
S31508004F3C23F003035360536843F0020353604B6832
S31508004F4C03F00C03082BFAD1C3E700BF001002408C
S31508004F5C0000FFF800ED00E00020024000224FF4AC
S31508004F6C1F0500B5504B85B00192029219684F4A3D
S31508004F7C41F001011960596840F2DC540A405A6044
S31508004F8C1A68184622F0847222F480321A601A685B
S31508004F9C22F480221A605A6822F4FE025A609D6036
S31508004FAC1A6842F480321A6002E0019BA34209D0C7
S31508004FBC036803F400330293019B01330193029BAC
S31508004FCC002BF2D0384B1B689A0368D5384A364BF7
S31508004FDC1068194640F010001060106820F00300A5
S31508004FEC1060106840F0020010605A685A605A68DF
S31508004FFC42F400525A605A6842F480625A605A68FF
S3150800500C22F47C125A605A6842F4E8125A601A68FA
S3150800501C42F080721A600B689B01FCD54A68224BD9
S3150800502C22F003024A604A6842F002024A605A6851
S3150800503C02F00C02082AFAD101255A68294622F4EC
S3150800504C80025A60DA69042042F40002DA61FEF73B
S3150800505C89FB0326482304AC24F8045D214615482D
S3150800506C8DF80F308DF80E60FEF714FB29460420D8
S3150800507CFEF778FB2025102321460E488DF80F30B5
S3150800508C8DF80E60ADF80C50FEF704FB294609485E
S3150800509CFEF766FBFBF71CFDFBF72CFDFCE76F2107
S315080050AC0548FBF7DDFC91E7001002400000FFF80D
S315080050BC00200240000801405C5B0008DFF834D091
S315080050CC002103E00C4B5B58435004310B480C4B46
S315080050DC42189A42F6D30B4A02E0002342F8043BE4
S315080050EC094B9A42F9D3FFF7B7FE00F03BF9FFF7E5
S315080050FC35FF704700500020245D00080000002092
S3150800510CC0020020C0020020AC130020FEE70000FD
S3150800511CFBF714BCFBF75CBC034B1B68052B00D0D8
S3150800512C7047FBF70BBC00BF6C130020174970B512
S3150800513C0B68174C9BB2174D238022882B881A4074
S3150800514C900516D422881A4012040ED4228802F42A
S3150800515C8062134200D170BD4FF6FF31BDE8704036
S3150800516C0A4A0D4B11605B681847FFF715F82B8830
S3150800517CECE74FF6FF53094A0B6013780133DBB2A1
S3150800518C1370FFF7C9FF2B88DCE700BF445C0040AF
S3150800519CAA130020A4130020700000206813002016
S315080051AC034B9B7A13B10522024B1A60704700BF5A
S315080051BC801300206C1300200422014B1A607047E0
S315080051CC6C130020704700BF062801D002207047D8
S315080051DC0B4B1B681A7802F07F02012AF6D110B520
S315080051EC5C7954B99A78212A07D1064A5C829A6165
S315080051FC204600F097F8204610BD022010BD00BFCF
S3150800520CA0130020315300080220704709B1022070
S3150800521C7047002814BF02200020704710B50024E0
S3150800522CFBF7FEFB044B1B689C7200F083F8FFF738
S3150800523CCBF9024B1C6010BDA01300206C13002088
S3150800524C10B50024254B264A1B68D2799C725A72D3
S3150800525CDC722046FFF784F820464FF40071FFF7FE
S3150800526C87F820461021FFF791F820464021FFF7D2
S3150800527C71F980212046FFF75BF92046FFF7F2F813
S3150800528C184B204693F82C10FFF720F92046FFF709
S3150800529CC5F821460120FFF76BF84FF48071012001
S315080052ACFFF746F9C0210120FFF754F940210120E8
S315080052BCFFF7FEF840210120FFF708F94FF440519B
S315080052CC0120FFF77DF820210120FFF75FF8204623
S315080052DCFEF724FF0122044B1A6010BDA013002010
S315080052EC685B0008700000206C1300200149FEF76B
S315080052FC69BC00BF680000200149FEF763BC00BF0B
S3150800530C60000020054B1B68DB78052B04D8044984
S3150800531C01EBC301FEF756BC00207047A013002012
S3150800532CA40000200149FEF74DBC00BF5800002020
S3150800533C704700BF38B50120FEF7C8F800224FF4B5
S3150800534CE0510120044B054D054C18601A601046B7
S3150800535C2A602180196038BD405C0040445C0040DE
S3150800536CA413002070B500250C4E0D4CA41BA410DC
S3150800537CA54209D100F050F800250A4E0A4CA41B88
S3150800538CA410A54205D170BD56F8253098470135AD
S3150800539CEEE756F8253098470135F2E71C5D00080C
S315080053AC1C5D00081C5D0008205D0008044B054ABE
S315080053BC1B681B6A002B08BF1346D3F8EC00704712
S315080053CC5C020020F000002082B001B901A942B1AC
S315080053DC4BB113780B601278101C18BF012002B061
S315080053EC70471046FBE76FF00100F8E703460244E6
S315080053FC934200D1704703F8011BF9E749B1FF2A1C
S3150800540C8BBF8A230A700360012088BF4FF0FF30D8
S3150800541C7047084670470000F8B500BFF8BC08BCD2
S3150800542C9E467047F8B500BFF8BC08BC9E46704748
S3150800543C006000080020000003000000008000083F
S3150800544C002000000400000000A000080020000056
S3150800545C0500000000C0000800200000060000003F
S3150800546C00E000080020000007000000000001080A
S3150800547C00200000080000000020010800200000A1
S3150800548C0900000000400108002000000A00000086
S3150800549C00600108002000000B00000000800108D5
S315080054AC002000000C00000000A0010800200000ED
S315080054BC0D00000000C00108002000000E000000CE
S315080054CC00E00108002000000F0000002E2E2F2EF1
S315080054DC2E2F2E2E2F2E2E2F536F757263652F415E
S315080054EC524D434D335F53544D333246312F7573FA
S315080054FC622E6300000008003F000000303A0000EE
S3150800550C2E2E2F2E2E2F2E2E2F2E2E2F536F7572AC
S3150800551C63652F66696C652E630000004669726DBB
S3150800552C7761726520757064617465207265717532
S3150800553C6573742064657465637465640A0D00008C
S3150800554C4F70656E696E67206669726D77617265F4
S3150800555C2066696C6520666F722072656164696E77
S3150800556C672E2E2E000000004552524F520A0D008F
S3150800557C4F4B0A0D000000005374617274696E6714
S3150800558C207468652070726F6772616D6D696E67DD
S3150800559C2073657175656E63650A0D0050617273CB
S315080055AC696E67206669726D776172652066696CCB
S315080055BC6520746F20646574656374206572617305
S315080055CC6520626C6F636B732E2E2E0045726173A9
S315080055DC696E672000000000206279746573206686
S315080055EC726F6D206D656D6F7279206174203078DD
S315080055FC0000000052656164696E67206C696E650F
S3150800560C2066726F6D2066696C652E2E2E45525279
S3150800561C4F520A0D00000000496E76616C696420D1
S3150800562C636865636B73756D20666F756E642E2E75
S3150800563C2E4552524F520A0D0000000050726F67E9
S3150800564C72616D6D696E67200000000020627974C6
S3150800565C657320746F206D656D6F72792061742087
S3150800566C3078000057726974696E672070726F67BC
S3150800567C72616D20636865636B73756D2E2E2E00D3
S3150800568C436C6F73696E67206669726D77617265B4
S3150800569C2066696C650A0D004669726D77617265DC
S315080056AC20757064617465207375636365737366BE
S315080056BC756C6C7920636F6D706C657465640A0D16
S315080056CC00000000809A45418E418F80454545492A
S315080056DC49498E8F9092924F994F555559999A9B45
S315080056EC9C9D9E9F41494F55A5A5A6A7A8A9AAABBF
S315080056FCACADAEAFB0B1B2B3B4B5B6B7B8B9BABB58
S3150800570CBCBDBEBFC0C1C2C3C4C5C6C7C8C9CACB47
S3150800571CCCCDCECFD0D1D2D3D4D5D6D7D8D9DADB37
S3150800572CDCDDDEDFE0E1E2E3E4E5E6E7E8E9EAEB27
S3150800573CECEDEEEFF0F1F2F3F4F5F6F7F8F9FAFB17
S3150800574CFCFDFEFF01030507090E10121416181CA2
S3150800575C1E000000222A3A3C3E3F7C7F00000000D7
S3150800576C2B2C3B3D5B5D0000C700FC00E900E2000A
S3150800577CE400E000E500E700EA00EB00E800EF00D3
S3150800578CEE00EC00C400C500C900E600C600F40033
S3150800579CF600F200FB00F900FF00D600DC00A200C0
S315080057ACA300A500A7209201E100ED00F300FA0082
S315080057BCF100D100AA00BA00BF001023AC00BD004E
S315080057CCBC00A100AB00BB009125922593250225B0
S315080057DC24256125622556255525632551255725EA
S315080057EC5D255C255B251025142534252C251C25C3
S315080057FC00253C255E255F255A25542569256625F1
S3150800580C602550256C256725682564256525592549
S3150800581C5825522553256B256A2518250C258825C8
S3150800582C84258C2590258025B103DF009303C003BE
S3150800583CA303C303B500C403A6039803A903B403BF
S3150800584C1E22C603B50329226122B10065226422F1
S3150800585C20232123F7004822B0001922B7001A2268
S3150800586C7F20B200A025A00061001A03E0001703F0
S3150800587CF8000703FF00010078010001300132012E
S3150800588C0601390110014A012E0179010601800130
S3150800589C4D00430281018201820184018401860143
S315080058AC8701870189018A018B018B018D018E0184
S315080058BC8F0190019101910193019401F6019601D2
S315080058CC9701980198013D029B019C019D012002BC
S315080058DC9F01A001A001A201A201A401A401A60195
S315080058ECA701A701A901AA01AB01AC01AC01AE0144
S315080058FCAF01AF01B101B201B301B301B501B501F5
S3150800590CB701B801B801BA01BB01BC01BC01BE01A3
S3150800591CF701C001C101C201C301C401C501C4011B
S3150800592CC701C801C701CA01CB01CA01CD011001C3
S3150800593CDD0101008E01DE011201F3010300F10104
S3150800594CF401F401F8012801220212013A020900B5
S3150800595C652C3B023B023D02662C3F02400241028B
S3150800596C410246020A015302400081018601550292
S3150800597C89018A0158028F015A0290015C025D0264
S3150800598C5E025F029301610262029401640265027F
S3150800599C66026702970196016A02622C6C026D0216
S315080059AC6E029C01700271029D01730274029F01C2
S315080059BC76027702780279027A027B027C02642CE0
S315080059CC7E027F02A60181028202A9018402850257
S315080059DC86028702AE014402B101B20145028D026C
S315080059EC8E028F0290029102B7017B030300FD031E
S315080059FCFE03FF03AC0304008603880389038A03AA
S31508005A0CB1031103C2030200A303A303C4030803CF
S31508005A1CCC0303008C038E038F03D8031801F203FF
S31508005A2C0A00F903F303F403F503F603F703F70384
S31508005A3CF903FA03FA033004200350041007600430
S31508005A4C22018A043601C1040E01CF040100C004E8
S31508005A5CD004440161052604000000007D1D0100E8
S31508005A6C632C001E9601A01E5A01001F0806101F63
S31508005A7C0606201F0806301F0806401F0606511F7B
S31508005A8C0700591F521F5B1F541F5D1F561F5F1FB0
S31508005A9C601F0806701F0E00BA1FBB1FC81FC91F40
S31508005AACCA1FCB1FDA1FDB1FF81FF91FEA1FEB1FD4
S31508005ABCFA1FFB1F801F0806901F0806A01F080662
S31508005ACCB01F0400B81FB91FB21FBC1FCC1F0100A2
S31508005ADCC31FD01F0206E01F0206E51F0100EC1FBC
S31508005AECF21F0100FC1F4E21010032217021100209
S31508005AFC842101008321D0241A05302C2F04602C14
S31508005B0C0201672C0601752C0201802C6401002DFC
S31508005B1C260841FF1A0300004F70656E424C54006C
S31508005B2C2F626F6F746C6F672E74787400000000A8
S31508005B3C2F64656D6F70726F675F6F6C696D6578D2
S31508005B4C696E6F5F73746D33322E73726563000002
S31508005B5C2E2E2F6D61696E2E63000000090220003F
S31508005B6C010100C0320904000002FF000004070509
S31508005B7C81024000000705010240000012011001D5
S31508005B8C00000040501DAC6000010102030100003A
S31508005B9C2C03570069006E00550053004200200084
S31508005BAC420075006C006B00200049006E00740002
S31508005BBC6500720066006100630065000403090451
S31508005BCC2603570069006E0055005300420020005A
S31508005BDC420075006C006B002000440065007600DE
S31508005BEC69006300650000001A034F007000650029
S31508005BFC6E0042004C0054002000550073006500EE
S31508005C0C72004300504F534958002E0000202020A4
S31508005C1C2020202020202828282828202020202042
S31508005C2C2020202020202020202020202088101012
S31508005C3C101010101010101010101010100404046E
S31508005C4C040404040404041010101010101041412C
S31508005C5C414141410101010101010101010101011A
S31508005C6C010101010101010110101010101042422E
S31508005C7C42424242020202020202020202020202EA
S31508005C8C020202020202020210101010200000008A
S31508005C9C00000000000000000000000000000000EA
S31508005CAC00000000000000000000000000000000DA
S31508005CBC00000000000000000000000000000000CA
S31508005CCC00000000000000000000000000000000BA
S31508005CDC00000000000000000000000000000000AA
S31508005CEC000000000000000000000000000000009A
S31508005CFC000000000000000000000000000000008A
S31508005D0C0000000000000000000000000000000079
S30908005D1C310100083B
S30908005D200D0100085B
S31508005D24040100001C0353004500520031003200F0
S31508005D3433003400350036003700380039003000A7
S31508005D441D510008694100086941000869410008B5
S31508005D5469410008694100086941000821510008A1
S31508005D646941000869410008694100086941000859
S31508005D7469410008694100087A5B000809000000C7
S31508005D84685B000820000000885B00081200000019
S31508005D94295200084D5200083D530008D151000805
S31508005DA4D55100081552000819520008F95200087E
S31508005DB405530008115300080000000040000000C5
S31508005DC403010000C85B000804000000F45B000837
S31508005DD41A000000CC5B000826000000040000201E
S31508005DE41C0000009C5B00082C00000069410008A8
S31508005DF4AD51000869410008694100086941000875
S31508005E04694100086941000869410008C55100084C
S31508005E14430000000000000000000000000000002D
S31508005E240000000000000000000000000000000060
S31508005E34430000000000000000000000000000000D
S31508005E440000000000000000000000000000000040
S31508005E5443000000000000000000000000000000ED
S31508005E640000000000000000000000000000000020
S31508005E7443000000000000000000000000000000CD
S31508005E840000000000000000000000000000000000
S31508005E9443000000000000000000000000000000AD
S31508005EA400000000000000000000000000000000E0
S31508005EB4430000000000000000000000000000008D
S31508005EC400000000000000000000000000000000C0
S31508005ED4430000000000000000000000000000006D
S31508005EE400000000000000000000000000000000A0
S31508005EF409540008D553000800000000185C00087F
S31508005F04165C0008175C0008175C0008175C000894
S31508005F14175C0008175C0008175C0008175C000883
S31508005F24175C0008175C0008FFFFFFFFFFFFFFFF71
S31508005F34FFFFFFFFFFFF00000100415343494900EB
S31508005F44000000000000000000000000000000003F
S31508005F5400000000000000000000415343494900C6
S31508005F64000000000000000000000000000000001F
S31508005F74000000000000000000000000600200208D
S31508005F8400000000000000000000000000000000FF
S31508005F9400000000000000000000000000000000EF
S31508005FA400000000000000000000000000000000DF
S31508005FB400000000000000000000000000000000CF
S31508005FC400000000000000000000000000000000BF
S31508005FD400000000000000000000000000000000AF
S705080050C9D9
